:0400000002099A3225
:01000B0032C2
:0100130032BA
:01001B0032B2
:0100230032AA
:01002B0032A2
:10099A0075810712090EE5826003020033020033F3
:100033001207C180FEC2A7D2A7227A327B001ABA66
:10004300FF011BEA4B70F722AA82AB837C007D0081
:10005300C3EC9AED64808BF063F08095F0501AC086
:1000630002C003C004C00512003DD005D004D00374
:10007300D0020CBC00DA0D80D7227A017B001ABAB9
:10008300FF011BEA4B70F7227A147B001ABAFF01B7
:100093001BEA4B70F7223098FDC2988599821200B3
:1000A300B1859982223098FDC29885998222AA82CD
:1000B3003099FDC2998A9922AA82AB83ACF07D0064
:1000C3008D060DEE2AF582E43BF5838CF01209725E
:1000D300FE8E07BE000280178F82C002C003C004D9
:1000E300C0051200B1D005D004D003D00280D122C4
:1000F3007A467B087C028A828B838CF01200BB22B7
:10010300AA37BA0D127A0C7B087C028A828B838C05
:10011300F01200BB1200F3227A007B008A04BC0AAF
:1001230002802E758211C002C0031200B1D003D029
:1001330002C002C003120099AC82D003D0028C0229
:100143008A04BC0D027A0AEB2442A8E0A6020B80C3
:10015300CB1BEB2442A8E076007A007B007C00EC0A
:100163002442F88605BD00028037E4F54F754E0A38
:100173008A828B83C002C003C004C0051208EFAE9D
:1001830082AF83D005D004D003D002ED3395E0F8DD
:10019300ED2EFEE83FFFEE24D0FAEF34FFFB0C8098
:1001A300BE8A828B8322309809120099AA828A37E9
:1001B30080037537FF227A4B7B087C028A828B830C
:1001C3008CF01200BB1200F322AA82C374099A4076
:1001D3000F74302AFB8B82C0021200B1D002800957
:1001E30074372AFA8A821200B122AA8274F05AFB67
:1001F300C4540FFB8B82C002C0031201CCD003D0C6
:1002030002740F5AFB8B821201CC22AA82AB838B1E
:10021300047D008C82C002C0031201EDD003D00222
:100223008A821201ED22AA82AB83754E10754F2785
:100233008A828B83C002C0031208B0AC82AD83D024
:1002430003D00274302CFCE43DFD8C48754E1075D0
:100253004F278A828B83120912AA82AB83754EE8D9
:10026300754F038A828B83C002C0031208B0AC822D
:10027300AD83D003D00274302CFCE43DFD8C497572
:100283004EE8754F038A828B83C002C003120912A2
:10029300AC82AD83D003D0028C028D03E4F54F759D
:1002A3004E648A828B83C002C0031208B0AC82AD55
:1002B30083D003D00274302CFCE43DFD8C4AE4F57A
:1002C3004F754E648A828B83C002C003120912AC3D
:1002D30082AD83D003D0028C028D03E4F54F754EBB
:1002E3000A8A828B83C002C0031208B0AC82AD833A
:1002F300D003D00274302CFCE43DFD8C4BE4F54F6D
:10030300754E0A8A828B83C002C003120912AC8223
:10031300AD83D003D0028C028D03E4F54F754E0AF2
:100323008A828B83C002C003120912AC82AD83D0D0
:1003330003D00274302CFCE43DFD8C4C7C007D002A
:10034300EC2448F88606BE3010C3EC9405ED940007
:1003530050070CBC00EA0D80E78C028D03BC050B33
:10036300BD0008EC24FFFAED34FFFB8A048B050A79
:10037300BA00010BEC2448F88682C002C0031200C5
:10038300B1D003D002C3EA9405EB940040DD2230E0
:1003930098091200A8AA828A3780037537FF2212B0
:1003A3000392AA82AB83BA1310BB000D120392AA65
:1003B30082AB83BA11F6BB00F322C2A790012C12C1
:1003C300004BD2A722E537B46527D2B3D2B4C2B566
:1003D300D2B2C2B6C2B7D2A712007DC2B390012C6B
:1003E30012004B1203BD90012C12004BD2B3120129
:1003F300B922E537B477028003020485D2B3C2B4CD
:10040300D2B5D2B2D2B6D2B7D2A712007DE536B4F6
:10041300FF02C2B390012C12004BE4F53BF53AE422
:10042300F531F530AA30AB31C3EA953CEB953D503D
:10043300467582111200B18530388531398538907F
:10044300AA397B004302808AA012007D1200A8AA69
:10045300828A807582131200B1AA807B00EA253A52
:10046300F53AEB353BF53B12003812008B0530E4CF
:10047300B53002053180ADD2B39000C812004B12E3
:1004830001B922E537B472028003020507E4F53BA4
:10049300F53AD2B3D2A7C2B4D2B5C2B2D2B6D2B7AA
:1004A3007534317A007B00C3EA953CEB953D50519E
:1004B3008A388B39853890AC397D004304808CA011
:1004C300C2B5C002C00312007DD003D0027580FF05
:1004D300AC807D00EC253AF53AED353BF53B858064
:1004E30082C002C0031201EDD003D002D2B5C00214
:1004F300C0031203A2D003D0020ABA00010B020404
:10050300AA1201B922E580B4FF02800B75343005CD
:1005130040E4B54002054122E537B46C44C2B3D28E
:10052300A790012C12004BD2B7D2B6D2B2D2B5D219
:10053300B41203BD90000512004BC2B7C2B612003D
:100543007D1203BD90000512004BC2B5D2B2D2B6E4
:10055300C2B712007D1203BD90000512004B1201B9
:10056300B922E537B463267A517B087C028A828BF1
:10057300838CF01200BBE53AF4FAE53BF4FB74011B
:100583002AF582E43BF58312020E1201B922D2A7A7
:10059300D2B3C2B4D2B5C2B2C2B7C2B6753800754F
:1005A30039017590007A017B004302808AA0C2B5AD
:1005B30012007D7580FF858035D2B5E535B4FF1F08
:1005C300E4F5397538317590317A007B0043028048
:1005D3008AA0C2B512007D7580FF858035D2B5052E
:1005E30038E4B538020539853890AA397B004302CF
:1005F300808AA0C2B512007D7580FF7535527536AD
:10060300FF22120591E535B45102802AE535B45233
:10061300028033E535B45502803CE535B461028090
:100623001DE535B462028026E535B46502802FE509
:1006330035B4FF378030753E00753F10802D753E11
:1006430000753F108025753E00753F20801D753E67
:1006530000753F208015753E00753F50800D753E37
:1006630000753F508005E4F53FF53EE4F53BF53A70
:10067300E4F541F540D2A7D2B3C2B4D2B7D2B6D2D1
:10068300B57534317A007B00C3EA953EEB953F5054
:10069300428A388B39853890AC397D004304808C8D
:1006A300A0C2B5C002C00312007DD003D002758082
:1006B300FFAC807D00EC253AF53AED353BF53BC0C8
:1006C30002C003120508D003D002D2B50ABA000152
:1006D3000B80B522E537B4730E12011BAA82AB83DC
:1006E3008A3C8B3D1201B922E537B46702800302CD
:1006F3000790120605E535B4FF0302077E7A5E7B99
:10070300087C028A828B838CF01200BB85358212AF
:1007130001EDE536B4FF0F7A6E7B087C028A828B8B
:10072300838CF01200BBE536B4050F7A737B087C2B
:10073300028A828B838CF01200BB7A777B087C025F
:100743008A828B838CF01200BB85408285418312A1
:1007530002297A847B087C028A828B838CF01200C4
:10076300BB7A8B7B087C028A828B838CF01200BB62
:10077300853C82853D83120229800F7A9D7B087C0C
:10078300028A828B838CF01200BB1201B922E537F7
:10079300B4702A1206058535821201ED75822C127A
:1007A30000B185408285418312022975822C120093
:1007B300B1853C82853D831202291201B922E4F5F9
:1007C30031F530E4F53DF53C759852758920758D0A
:1007D300FDD28E1200997A0C7B087C028A828B836D
:1007E3008CF01200BB1200F31201A91201031206CE
:1007F300D71203C81203F512048612051B120565EE
:100803001206EB12079180E0220A0D2045617379ED
:100813002D446F776E6C6F616465722056322E3093
:1008230020666F722041544D454C20383953353181
:100833002F35322028736463632076657273696F82
:100843006E29000A0D203E000A0D206F6B000A0D71
:100853002043484B53554D203D20000A0D20666F21
:10086300756E6420746172676574002D31325600B1
:100873002D3556000A0D206E6F6E626C616E6B2013
:1008830000206279746573000A0D206279746573C0
:1008930020636F756E74657220000A0D204E6F74AD
:1008A30020666F756E6420383953787800AA82AB5E
:1008B300837C007D007E10EB235401FFEBCA25E00F
:1008C300CA33FBEDCC25E0CC33FDEF6003430401D9
:1008D300C3EC954EED954F400CC3EC954EFCED9556
:1008E3004FFD430201DED08A828B8322AA83AB822F
:1008F3008BF0E54EA4F8A9F08AF0E54EA429F98B14
:10090300F0E54FA429F5838882222275820022AA6A
:1009130082AB837C007D00E54F235401FE7028AE3B
:100923004EE54FCE25E0CE33FF8E4E8F4FC3EA9E6A
:10093300EB9F500E8E4EEFC313C54E13C54EF54FAE
:1009430080050D8D0480D0C3EA954EEB954F400989
:10095300C3EA954EFAEB954FFBE54FC313C54E1310
:10096300C54EF54F8C051CED70DD8A828B8322C842
:10097300C0E0E5F0600D14600F14600F1460107494
:10098300FF800FA882E6800AE08007E4938003A833
:0709930082E2F8D0E0C82267
:00000001FF
